:1000000000308A004E2900000A108A100A11820767
:1000100028340C34013406340A108A100A1182077D
:100020002034203420342E3400340A108A100A116F
:100030008207413454342B344334423443340D3436
:1000400000340A108A100A1182070C344F344434E9
:10005000503431343A342534733400340A108A1061
:100060000A1182070C344F344434503432343A3459
:100070002534733400340A108A100A1182070C34B4
:100080004F344434503433343A34253473340034E8
:100090000A108A100A1182070C344F344434503449
:1000A00034343A342534733400340A108A100A1177
:1000B00082070C344F344434503435343A342534C8
:1000C0007334003441308400831700080319792801
:1000D0000130F800BF30F7006400F70B6C28F80B14
:1000E0006A284A30F700F70B732800006400800B81
:1000F000682800340708F0390317C80047080F398B
:100100004804031387000614831606106400831244
:10011000061083160610831200340317C508031D4A
:100120009528031386109728031703138614831644
:10013000861083120317C60E4608C70003137A20E1
:100140000317C60E4608C70003137A2064000C305C
:10015000F700F70BA928AC28003414300317C100AE
:1001600003136220F03083168705831286108316EE
:100170008610831206108316061083120317BD0122
:100180003D08023C031CD0280230C100031362204A
:1001900003300317C70003137A200317BD0AC028D2
:1001A00064000C30F700F70BD328D6280230C700C4
:1001B00003137A2064000C30F700F70BDD28E028E9
:1001C0000317BD013D08023C031CF8283D0803133A
:1001D00004200317BE00C5013E08C60003138D208E
:1001E00002300317C100031362200317BD0AE2287F
:1001F00003139029013003174102C3004208023C57
:10020000031D04294030C30743088038C400C501DA
:100210004408C60003138D200034031740080C3A2D
:10022000031303191D29063A03192929073A03194B
:100230003129053A031938293F290317C50101302F
:10024000C60003138D2002300317C1000313622080
:100250004D2901300317C1000230C2000313FA20F8
:100260004D2901300317C100C2000313FA204D29A4
:100270000317C5011030C60003138D204D29031745
:1002800040081F3C031C46290730C0050130C5004B
:100290004008C60003138D204D29003484018313C8
:1002A0001F3083050C3083169900A63098009030DB
:1002B0008312980083161F149F141F159F11073077
:1002C0009C00FF308312A00083161F149F141F157B
:1002D0009F1183121F108316091283129412A01209
:1002E00020088316870083122016200883168700B3
:1002F0008312A01120088316870000308312940017
:10030000831694000108C7390838810083129001D0
:100310000030F80092000030831692008312AD285E
:100320000830E200FA300317C10003136220E20B29
:1003300092290C300317C00003130D21203003173E
:10034000C00003130D215A300317C00003130D2101
:1003500064300317C1000313622061300317C0002B
:1003600003130D2132300317C100031362207630CE
:100370000317C00003130D2132300317C10003130C
:10038000622061300317C00003130D2132300317C0
:10039000C1000313622064300317C00003130D2152
:1003A00032300317C1000313622069300317C00005
:1003B00003130D2132300317C100031362206D3087
:1003C0000317C00003130D2132300317C1000313BC
:1003D000622020300317C00003130D2132300317B1
:1003E000C1000313622073300317C00003130D21F3
:1003F00032300317C1000313622079300317C000A5
:1004000003130D2132300317C10003136220733030
:100410000317C00003130D2132300317C10003136B
:10042000622074300317C00003130D21323003170C
:10043000C1000313622065300317C00003130D21B0
:1004400032300317C100031362206D300317C00060
:1004500003130D210A300317C00003130D2196303A
:100460000317C10003136220E20162080C20E20AB4
:10047000F7000317C00003130D2104306202031DAF
:10048000352A96300317C10003136220203003176A
:10049000C00003130D212E300317C00003130D21DC
:1004A000AF300317C1000313622020300317C000D0
:1004B00003130D212E300317C00003130D2102304A
:1004C000E20096300317C10003136220E20B612A99
:1004D00020300317C00003130D212E300317C00076
:1004E00003130D210230E200C8300317C1000313CB
:1004F0006220E20B742A20300317C00003130D2181
:100500002E300317C00003130D210530E2006E30BA
:100510000317C10003136220E20B872A831605121A
:10052000831205120630E200FA300317C1000313EC
:100530006220E20B942A8316051283120516E2014B
:1005400062081520E20AF70077080C1EA52A990018
:1005500007306202031DA02A213084008313840324
:10056000840A8C1EB12A1A0880000D300002031D77
:10057000B02A80014E30840083138403840A8C1EC9
:10058000BF2A1A0880000D300002031DBE2A800118
:10059000A030840083138403840A8C1ECD2A1A0899
:1005A00080000D300002031DCC2A800158308400E9
:1005B00083138403840A8C1EDB2A1A0880000D3002
:1005C0000002031DDA2A800110308400831784039F
:1005D000840A8C1EE92A1A0880000D300002031DCF
:1005E000E82A8001E20162082120E20AF7000317ED
:1005F000C00003130D2106306202031DF32A2130CF
:1006000084008313003000040319182BE40104084C
:10061000E3006410831B641400080317C000031375
:100620000D2163088400831364188317840A022B46
:100630000830E200FA300317C10003136220E20B16
:100640001A2BE20162082E20E20AF7000317C0000D
:1006500003130D2106306202031D222B4E3084004D
:100660008313003000040319472BE4010408E3005E
:100670006410831B641400080317C00003130D21CA
:1006800063088400831364188317840A312B0830AD
:10069000E200FA300317C10003136220E20B492B7A
:1006A000E20162083B20E20AF7000317C0000313CF
:1006B0000D2106306202031D512BA03084008313EC
:1006C000003000040319762BE4010408E3006410F1
:1006D000831B641400080317C00003130D21630873
:1006E0008400831364188317840A602B0830E200A7
:1006F000FA300317C10003136220E20B782BE201EA
:1007000062084820E20AF7000317C00003130D2116
:1007100006306202031D802B5830840083130030A2
:1007200000040319A52BE4010408E3006410831BF3
:10073000641400080317C00003130D21630884002C
:10074000831364188317840A8F2B0830E200FA3071
:100750000317C10003136220E20BA72BE20162081A
:100760005520E20AF7000317C00003130D210630DD
:100770006202031DAF2B1030840083170030000489
:100780000319D42BE4010408E3006410831B6414F0
:1007900000080317C00003130D21630884008313AE
:1007A00064188317840ABE2B831605128312051260
:1007B00096300317C10003136220831605128312BB
:1007C000051664300317C100031362208316051257
:1007D0008312051296300317C1000313622083169B
:1007E00005128312051664300317C100031362203B
:1007F000831605128312051296300317C1000313E6
:10080000622083160512831205160630E200FA30C4
:100810000317C10003136220E20B072C8E2A63002A
:02400E00393F38
:00000001FF
